:1000000012C0189518951895189518951895189563
:100010001895189518951895189518951895189578
:100020001895189518958FE58DBFC0E2E4ED4E2E1A
:1000300084E08EBFD4E0F3E05F2EEEEFF3E0A0E6C5
:10004000B0E088278D933197E9F785E089B980E0A2
:1000500080BD88E18AB96624B89A8F9A8E9A8D9A63
:10006000B99ABA98BB98BC9A81E080939D00C29AD5
:10007000C39A80E080939C00969882E390E053D3EB
:10008000969A82E390E04FD3969882E390E04BD328
:10009000969A82E390E047D39698C098959897985F
:1000A000A0E6B0E06CD344E650E060E070E0A0E68B
:1000B000B0E00D911D912D913C916CD314F009F09D
:1000C00004C0A0E6B0E0F0D2EECF8D9A8F9A979858
:1000D000ACE9B0E098E08D91983018F4392F992769
:1000E00002C038E098508795959808F4959A0000DA
:1000F0000000979AEF93FF93E2E0F0E00BD3FF91BB
:10010000EF919798EF93FF93E2E0F0E003D3FF9134
:10011000EF913A9541F79923F1F68D9A8F9A979836
:10012000ACE9B0E098E08D91983018F4392F992718
:1001300002C038E098508795959808F4959A000089
:100140000000979AEF93FF93E2E0F0E0E3D2FF9193
:10015000EF919798EF93FF93E2E0F0E0DBD2FF910D
:10016000EF913A9541F79923F1F68D9A8F9A9798E6
:10017000ACE9B0E098E08D91983018F4392F9927C8
:1001800002C038E098508795959808F4959A000039
:100190000000979AEF93FF93E2E0F0E0BBD2FF916B
:1001A000EF919798EF93FF93E2E0F0E0B3D2FF91E5
:1001B000EF913A9541F79923F1F68D9A8F9A979896
:1001C000ACE9B0E098E08D91983018F4392F992778
:1001D00002C038E098508795959808F4959A0000E9
:1001E0000000979AEF93FF93E2E0F0E093D2FF9143
:1001F000EF919798EF93FF93E2E0F0E08BD2FF91BD
:10020000EF913A9541F79923F1F6C09A000000006A
:1002100000000000C098000000008D9A8F9A979807
:10022000ACE9B0E098E08D91983018F4392F992717
:1002300002C038E098508795959808F4959A000088
:100240000000979AEF93FF93E2E0F0E063D2FF9112
:10025000EF919798EF93FF93E2E0F0E05BD2FF918C
:10026000EF913A9541F79923F1F68D9A8F9A9798E5
:10027000ACE9B0E098E08D91983018F4392F9927C7
:1002800002C038E098508795959808F4959A000038
:100290000000979AEF93FF93E2E0F0E03BD2FF91EA
:1002A000EF919798EF93FF93E2E0F0E033D2FF9164
:1002B000EF913A9541F79923F1F68D9A8F9A979895
:1002C000ACE9B0E098E08D91983018F4392F992777
:1002D00002C038E098508795959808F4959A0000E8
:1002E0000000979AEF93FF93E2E0F0E013D2FF91C2
:1002F000EF919798EF93FF93E2E0F0E00BD2FF913C
:10030000EF913A9541F79923F1F68D9A8F9A979844
:10031000ACE9B0E098E08D91983018F4392F992726
:1003200002C038E098508795959808F4959A000097
:100330000000979AEF93FF93E2E0F0E0EBD1FF919A
:10034000EF919798EF93FF93E2E0F0E0E3D1FF9114
:10035000EF913A9541F79923F1F6C09A0000000019
:1003600000000000C09800000000A4E6B0E0E4E255
:10037000F8E0FBD18D9A8F9A9798A4E6B0E090E2CE
:100380008D91983018F4392F992702C038E0985091
:100390008795959808F4959A00000000979AEF9336
:1003A000FF93E2E0F0E0B6D1FF91EF919798EF93E1
:1003B000FF93E2E0F0E0AED1FF91EF913A9541F783
:1003C0009923F1F68D9A8F9A9798ADE9B0E098E06D
:1003D0008D91983018F4392F992702C038E0985041
:1003E0008795959808F4959A00000000979AEF93E6
:1003F000FF93E2E0F0E08ED1FF91EF919798EF93B9
:10040000FF93E2E0F0E086D1FF91EF913A9541F75A
:100410009923F1F6C09A0000000000000000C09887
:1004200000000000FCD1A8E7B0E03FE04ED1F4D1DD
:1004300041E050E060E070E0A8E7B0E0BED1BB274B
:10044000A0E10D911D912D913C91A4D109F002C024
:10045000969801C0969AE3D1A8E6B0E03FE035D186
:10046000DBD1DDD1A6EAB0E03FE02FD1D5D1D7D1A5
:10047000ACE8B0E03FE029D1CFD10000000000009F
:100480000000000000000000A8E6B0E096D1A4E65D
:10049000B0E00D931D932D933D93A6EAB0E08DD16E
:1004A000A2EAB0E00D931D932D933D93ACE8B0E02C
:1004B00084D1A8E8B0E00D931D932D933D93A0E661
:1004C000B0E0E8E2F8E051D1A2EAB0E04D915D91F0
:1004D0006D917C91A0E6B0E00D911D912D913C9124
:1004E00059D114F009F0DDC0A4E6B0E00D911D91E2
:1004F0002D913C91A8E8B0E04D915D916D917C917A
:1005000044D1A4E6B0E00D931D932D933D938D9AB5
:100510008F9A9798A4E6B0E090E28D91983018F405
:10052000392F992702C038E098508795959808F49C
:10053000959A00000000979AEF93FF93E2E0F0E0B5
:10054000E9D0FF91EF919798EF93FF93E2E0F0E00D
:10055000E1D0FF91EF913A9541F79923F1F68D9A09
:100560008F9A9798ADE9B0E098E08D91983018F4A3
:10057000392F992702C038E098508795959808F44C
:10058000959A00000000979AEF93FF93E2E0F0E065
:10059000C1D0FF91EF919798EF93FF93E2E0F0E0E5
:1005A000B9D0FF91EF913A9541F79923F1F6C09AAE
:1005B0000000000000000000C0980000EF93FF93CF
:1005C000E8E1F0E0A7D0FF91EF91AEE9B0E0D5D03F
:1005D000A0EAB0E0D2D080E092E0A6EBB0E08D934C
:1005E0009C93C198EF93FF93E8E1F0E093D0FF91E3
:1005F000EF91A6EBB0E00D911C91003050E0150793
:1006000010F009F001C035C0C498EF93FF93E8E102
:10061000F0E080D0FF91EF91B29B0EC0AEE9B0E068
:100620000D911C91A6EBB0E04D915C91040F151F4C
:10063000AEE9B0E00D931C93B39B0EC0A0EAB0E00E
:100640000D911C91A6EBB0E04D915C91040F151F2C
:10065000A0EAB0E00D931C93C49AEF93FF93E8E1F6
:10066000F0E058D0FF91EF9191E0A6EBB0E06AD0B6
:10067000C0CFC19AC49AEF93FF93E1E1F1E04AD071
:10068000FF91EF9132E0AEE9B0E03BD0000032E004
:10069000A0EAB0E036D000000000A0E6B0E004D050
:1006A00013CFC0CEF894FFCF0D911D912D913C91A9
:1006B00081E0080F8827181F281F381F3C932E93AE
:1006C0001E930E930895ACEBB3E017D08D3049F034
:1006D000883079F03323C9F38D933A9563FE16D0B1
:1006E000F4CF63FC03C012D08AE010D088278C932B
:1006F00008950CD011973395E8CF5F9BFECF8CB156
:1007000008958D9103D03A95E1F708955D9BFECF52
:100710008CB908953197F1F70895689462F80895B7
:10072000E89462F80895EF93FF93EE27E82BE92B06
:1007300031F0EDECFAE03197F1F70197D1F7FF9145
:10074000EF910895903041F00D911C911695079509
:100750009A95E1F71C930E930895C8953196002061
:10076000089591E005C092E003C094E001C098E0D4
:10077000F4DF0D929A95E1F7089582E001C084E0DC
:1007800099279D938A95E9F70895040F151F261F51
:10079000371F089504171507260737070895000F18
:1007A000111F221F331F0895009510952095309535
:1007B0000F5F1F4F2F4F3F4F08950027112722270C
:1007C00033271DD08A3328F4803318F005D015D094
:1007D000F9CF0EF4E9CF089580538F93402F512F16
:1007E000622F732FDCDFDBDFD0DFD9DF8F9199271A
:1007F000080F191F291F391F08958D910895E89436
:10080000FCDF8032E9F38B32D9F38930C9F38D32C2
:1008100011F46894F2CF0895E89463F80895689409
:0C08200063F8089500366E01010000002E
:00000001FF
